 j2pcsc

 Timestamp is ffffffff (Sun Feb  7 06:28:15 2106)

 Preferred load address is 10000000

 Start         Length     Name                   Class
 0001:00000000 00001546H .text$mn                CODE
 0002:00000000 000000b0H .idata$5                DATA
 0002:000000b0 00000004H .00cfg                  DATA
 0002:000000b4 00000004H .CRT$XCA                DATA
 0002:000000b8 00000004H .CRT$XCZ                DATA
 0002:000000bc 00000004H .CRT$XIA                DATA
 0002:000000c0 00000004H .CRT$XIZ                DATA
 0002:000000c4 00000004H .CRT$XPA                DATA
 0002:000000c8 00000004H .CRT$XPZ                DATA
 0002:000000cc 00000004H .CRT$XTA                DATA
 0002:000000d0 00000008H .CRT$XTZ                DATA
 0002:000000d4 00000000H .gfids$y                DATA
 0002:000000d8 000001a0H .rdata                  DATA
 0002:00000278 00000004H .rdata$sxdata           DATA
 0002:0000027c 00000284H .rdata$zzzdbg           DATA
 0002:00000500 00000004H .rtc$IAA                DATA
 0002:00000504 00000004H .rtc$IZZ                DATA
 0002:00000508 00000004H .rtc$TAA                DATA
 0002:0000050c 00000004H .rtc$TZZ                DATA
 0002:00000510 00000090H .xdata$x                DATA
 0002:000005a0 000002e0H .edata                  DATA
 0002:00000880 00000078H .idata$2                DATA
 0002:000008f8 00000014H .idata$3                DATA
 0002:0000090c 000000b0H .idata$4                DATA
 0002:000009bc 00000394H .idata$6                DATA
 0003:00000000 00000018H .data                   DATA
 0003:00000018 00000374H .bss                    DATA
 0004:00000000 00000060H .rsrc$01                DATA
 0004:00000060 00000320H .rsrc$02                DATA

  Address         Publics by Value              Rva+Base       Lib:Object

 0000:00000000       ___x64_code_ranges_to_entry_points 00000000     <absolute>
 0000:00000000       ___volatile_metadata       00000000     <absolute>
 0000:00000000       ___arm64x_native_entrypoint 00000000     <absolute>
 0000:00000000       ___hybrid_code_map         00000000     <absolute>
 0000:00000000       ___guard_longjmp_count     00000000     <absolute>
 0000:00000000       ___arm64x_redirection_metadata_count 00000000     <absolute>
 0000:00000000       ___dynamic_value_reloc_table 00000000     <absolute>
 0000:00000000       ___guard_iat_table         00000000     <absolute>
 0000:00000000       ___hybrid_auxiliary_iat    00000000     <absolute>
 0000:00000000       ___hybrid_code_map_count   00000000     <absolute>
 0000:00000000       ___guard_longjmp_table     00000000     <absolute>
 0000:00000000       ___AbsoluteZero            00000000     <absolute>
 0000:00000000       ___guard_fids_count        00000000     <absolute>
 0000:00000000       ___enclave_config          00000000     <absolute>
 0000:00000000       ___guard_eh_cont_count     00000000     <absolute>
 0000:00000000       ___x64_code_ranges_to_entry_points_count 00000000     <absolute>
 0000:00000000       ___guard_iat_count         00000000     <absolute>
 0000:00000000       ___arm64x_redirection_metadata 00000000     <absolute>
 0000:00000000       ___guard_eh_cont_table     00000000     <absolute>
 0000:00000000       ___arm64x_extra_rfe_table_size 00000000     <absolute>
 0000:00000000       ___arm64x_extra_rfe_table  00000000     <absolute>
 0000:00000000       ___guard_fids_table        00000000     <absolute>
 0000:00000001       ___safe_se_handler_count   00000001     <absolute>
 0000:00000100       ___guard_flags             00000100     <absolute>
 0000:00000000       ___ImageBase               10000000     <linker-defined>
 0001:00000000       _JNI_OnLoad@8              10001000 f   pcsc.obj
 0001:00000008       _Java_sun_security_smartcardio_PCSC_SCardBeginTransaction@16 10001008 f   pcsc.obj
 0001:00000020       _Java_sun_security_smartcardio_PCSC_SCardConnect@28 10001020 f   pcsc.obj
 0001:00000089       _Java_sun_security_smartcardio_PCSC_SCardControl@24 10001089 f   pcsc.obj
 0001:0000016c       _Java_sun_security_smartcardio_PCSC_SCardDisconnect@20 1000116c f   pcsc.obj
 0001:00000188       _Java_sun_security_smartcardio_PCSC_SCardEndTransaction@20 10001188 f   pcsc.obj
 0001:000001a4       _Java_sun_security_smartcardio_PCSC_SCardEstablishContext@12 100011a4 f   pcsc.obj
 0001:000001d7       _Java_sun_security_smartcardio_PCSC_SCardGetStatusChange@32 100011d7 f   pcsc.obj
 0001:000003c3       _Java_sun_security_smartcardio_PCSC_SCardListReaders@16 100013c3 f   pcsc.obj
 0001:0000044e       _Java_sun_security_smartcardio_PCSC_SCardStatus@20 1000144e f   pcsc.obj
 0001:00000549       _Java_sun_security_smartcardio_PCSC_SCardTransmit@32 10001549 f   pcsc.obj
 0001:00000644       _handleRV                  10001644 f   pcsc.obj
 0001:00000660       _pcsc_multi2jstring        10001660 f   pcsc.obj
 0001:00000741       _throwOutOfMemoryError     10001741 f   pcsc.obj
 0001:00000762       _throwPCSCException        10001762 f   pcsc.obj
 0001:000007ae       _SCardEstablishContext@16  100017ae f   winscard:WinSCard.dll
 0001:000007b4       _SCardListReadersA@16      100017b4 f   winscard:WinSCard.dll
 0001:000007ba       _SCardGetStatusChangeA@16  100017ba f   winscard:WinSCard.dll
 0001:000007c0       _SCardConnectA@24          100017c0 f   winscard:WinSCard.dll
 0001:000007c6       _SCardDisconnect@8         100017c6 f   winscard:WinSCard.dll
 0001:000007cc       _SCardBeginTransaction@4   100017cc f   winscard:WinSCard.dll
 0001:000007d2       _SCardEndTransaction@8     100017d2 f   winscard:WinSCard.dll
 0001:000007d8       _SCardStatusA@28           100017d8 f   winscard:WinSCard.dll
 0001:000007de       _SCardTransmit@28          100017de f   winscard:WinSCard.dll
 0001:000007e4       _SCardControl@28           100017e4 f   winscard:WinSCard.dll
 0001:000007ea       @__security_check_cookie@4 100017ea f   MSVCRT:secchk.obj
 0001:00000800       __chkstk                   10001800 f   MSVCRT:chkstk.obj
 0001:00000800       __alloca_probe             10001800 f   MSVCRT:chkstk.obj
 0001:00000b6d       __DllMainCRTStartup@12     10001b6d f   MSVCRT:dll_dllmain.obj
 0001:00000b90       ___raise_securityfailure   10001b90 f   MSVCRT:gs_report.obj
 0001:00000bb8       ___report_gsfailure        10001bb8 f   MSVCRT:gs_report.obj
 0001:00000cfe       ___security_init_cookie    10001cfe f   MSVCRT:gs_support.obj
 0001:00000d49       _DllMain@12                10001d49 f   MSVCRT:dll_dllmain_stub.obj
 0001:00000d6b       ?__scrt_initialize_type_info@@YAXXZ 10001d6b f   MSVCRT:tncleanup.obj
 0001:00000d77       ?__scrt_uninitialize_type_info@@YAXXZ 10001d77 f   MSVCRT:tncleanup.obj
 0001:00000d83       ___local_stdio_printf_options 10001d83 f i MSVCRT:default_local_stdio_options.obj
 0001:00000d89       ___local_stdio_scanf_options 10001d89 f i MSVCRT:default_local_stdio_options.obj
 0001:00000d8f       ___scrt_initialize_default_local_stdio_options 10001d8f f   MSVCRT:default_local_stdio_options.obj
 0001:00000df0       ___scrt_acquire_startup_lock 10001df0 f   MSVCRT:utility.obj
 0001:00000e22       ___scrt_dllmain_after_initialize_c 10001e22 f   MSVCRT:utility.obj
 0001:00000e4d       ___scrt_dllmain_before_initialize_c 10001e4d f   MSVCRT:utility.obj
 0001:00000e5b       ___scrt_dllmain_crt_thread_attach 10001e5b f   MSVCRT:utility.obj
 0001:00000e7a       ___scrt_dllmain_crt_thread_detach 10001e7a f   MSVCRT:utility.obj
 0001:00000e87       ___scrt_dllmain_exception_filter 10001e87 f   MSVCRT:utility.obj
 0001:00000ebb       ___scrt_dllmain_uninitialize_c 10001ebb f   MSVCRT:utility.obj
 0001:00000ede       ___scrt_dllmain_uninitialize_critical 10001ede f   MSVCRT:utility.obj
 0001:00000eeb       ___scrt_initialize_crt     10001eeb f   MSVCRT:utility.obj
 0001:00000f24       ___scrt_initialize_onexit_tables 10001f24 f   MSVCRT:utility.obj
 0001:00000fab       ___scrt_is_nonwritable_in_current_image 10001fab f   MSVCRT:utility.obj
 0001:0000103f       ___scrt_release_startup_lock 1000203f f   MSVCRT:utility.obj
 0001:0000105c       ___scrt_uninitialize_crt   1000205c f   MSVCRT:utility.obj
 0001:00001084       ___scrt_get_dyn_tls_init_callback 10002084 f   MSVCRT:dyn_tls_init.obj
 0001:0000108a       ___scrt_fastfail           1000208a f   MSVCRT:utility_desktop.obj
 0001:000011a4       __crt_debugger_hook        100021a4 f   MSVCRT:utility_desktop.obj
 0001:000011ac       __RTC_Initialize           100021ac f   MSVCRT:initsect.obj
 0001:000011d8       __RTC_Terminate            100021d8 f   MSVCRT:initsect.obj
 0001:00001210       __SEH_prolog4              10002210 f   MSVCRT:sehprolg4.obj
 0001:00001254       __SEH_epilog4              10002254 f   MSVCRT:sehprolg4.obj
 0001:00001268       __except_handler4          10002268 f   MSVCRT:chandler4gs.obj
 0001:00001297       @_guard_check_icall_nop@4  10002297 f i MSVCRT:guard_support.obj
 0001:0000129a       ___isa_available_init      1000229a f   MSVCRT:cpu_disp.obj
 0001:0000146a       __get_startup_argv_mode    1000246a f   MSVCRT:argv_mode.obj
 0001:0000146e       ___scrt_is_ucrt_dll_in_use 1000246e f   MSVCRT:ucrt_detection.obj
 0001:0000147a       _IsProcessorFeaturePresent@4 1000247a f   kernel32:KERNEL32.dll
 0001:00001480       ___std_type_info_destroy_list 10002480 f   vcruntime:VCRUNTIME140.dll
 0001:00001486       _memset                    10002486 f   vcruntime:VCRUNTIME140.dll
 0001:0000148c       __except_handler4_common   1000248c f   vcruntime:VCRUNTIME140.dll
 0001:00001492       _strlen                    10002492 f   ucrt:api-ms-win-crt-string-l1-1-0.dll
 0001:00001498       __initterm                 10002498 f   ucrt:api-ms-win-crt-runtime-l1-1-0.dll
 0001:0000149e       __initterm_e               1000249e f   ucrt:api-ms-win-crt-runtime-l1-1-0.dll
 0001:000014a4       __seh_filter_dll           100024a4 f   ucrt:api-ms-win-crt-runtime-l1-1-0.dll
 0001:000014aa       __configure_narrow_argv    100024aa f   ucrt:api-ms-win-crt-runtime-l1-1-0.dll
 0001:000014b0       __initialize_narrow_environment 100024b0 f   ucrt:api-ms-win-crt-runtime-l1-1-0.dll
 0001:000014b6       __initialize_onexit_table  100024b6 f   ucrt:api-ms-win-crt-runtime-l1-1-0.dll
 0001:000014bc       __execute_onexit_table     100024bc f   ucrt:api-ms-win-crt-runtime-l1-1-0.dll
 0001:000014c2       __cexit                    100024c2 f   ucrt:api-ms-win-crt-runtime-l1-1-0.dll
 0001:000014c8       ___acrt_uninitialize       100024c8 f   MSVCRT:ucrt_stubs.obj
 0001:000014c8       ___vcrt_uninitialize       100024c8 f   MSVCRT:ucrt_stubs.obj
 0001:000014c8       ___acrt_thread_attach      100024c8 f   MSVCRT:ucrt_stubs.obj
 0001:000014c8       ___scrt_stub_for_acrt_initialize 100024c8 f   MSVCRT:ucrt_stubs.obj
 0001:000014c8       ___vcrt_thread_attach      100024c8 f   MSVCRT:ucrt_stubs.obj
 0001:000014c8       ___acrt_uninitialize_critical 100024c8 f   MSVCRT:ucrt_stubs.obj
 0001:000014c8       ___vcrt_thread_detach      100024c8 f   MSVCRT:ucrt_stubs.obj
 0001:000014c8       ___scrt_stub_for_acrt_uninitialize_critical 100024c8 f   MSVCRT:ucrt_stubs.obj
 0001:000014c8       ___acrt_thread_detach      100024c8 f   MSVCRT:ucrt_stubs.obj
 0001:000014c8       ___vcrt_initialize         100024c8 f   MSVCRT:ucrt_stubs.obj
 0001:000014c8       ___acrt_initialize         100024c8 f   MSVCRT:ucrt_stubs.obj
 0001:000014c8       ___scrt_stub_for_acrt_thread_detach 100024c8 f   MSVCRT:ucrt_stubs.obj
 0001:000014c8       ___vcrt_uninitialize_critical 100024c8 f   MSVCRT:ucrt_stubs.obj
 0001:000014c8       ___scrt_stub_for_acrt_thread_attach 100024c8 f   MSVCRT:ucrt_stubs.obj
 0001:000014c8       ___scrt_stub_for_acrt_uninitialize 100024c8 f   MSVCRT:ucrt_stubs.obj
 0001:000014cb       __is_c_termination_complete 100024cb f   MSVCRT:ucrt_stubs.obj
 0001:000014cb       ___scrt_stub_for_is_c_termination_complete 100024cb f   MSVCRT:ucrt_stubs.obj
 0001:000014ce       __filter_x86_sse2_floating_point_exception 100024ce f   MSVCRT:x86_exception_filter.obj
 0001:000014ce       __filter_x86_sse2_floating_point_exception_default 100024ce f   MSVCRT:x86_exception_filter.obj
 0002:00000000       __imp__IsProcessorFeaturePresent@4 10003000     kernel32:KERNEL32.dll
 0002:00000004       __imp__GetCurrentProcessId@0 10003004     kernel32:KERNEL32.dll
 0002:00000008       __imp__QueryPerformanceCounter@4 10003008     kernel32:KERNEL32.dll
 0002:0000000c       __imp__TerminateProcess@8  1000300c     kernel32:KERNEL32.dll
 0002:00000010       __imp__GetCurrentProcess@0 10003010     kernel32:KERNEL32.dll
 0002:00000014       __imp__IsDebuggerPresent@0 10003014     kernel32:KERNEL32.dll
 0002:00000018       __imp__InitializeSListHead@4 10003018     kernel32:KERNEL32.dll
 0002:0000001c       __imp__DisableThreadLibraryCalls@4 1000301c     kernel32:KERNEL32.dll
 0002:00000020       __imp__GetSystemTimeAsFileTime@4 10003020     kernel32:KERNEL32.dll
 0002:00000024       __imp__UnhandledExceptionFilter@4 10003024     kernel32:KERNEL32.dll
 0002:00000028       __imp__SetUnhandledExceptionFilter@4 10003028     kernel32:KERNEL32.dll
 0002:0000002c       __imp__GetCurrentThreadId@0 1000302c     kernel32:KERNEL32.dll
 0002:00000030       \177KERNEL32_NULL_THUNK_DATA 10003030     kernel32:KERNEL32.dll
 0002:00000034       __imp__memset              10003034     vcruntime:VCRUNTIME140.dll
 0002:00000038       __imp____std_type_info_destroy_list 10003038     vcruntime:VCRUNTIME140.dll
 0002:0000003c       __imp___except_handler4_common 1000303c     vcruntime:VCRUNTIME140.dll
 0002:00000040       \177VCRUNTIME140_NULL_THUNK_DATA 10003040     vcruntime:VCRUNTIME140.dll
 0002:00000044       __imp__SCardTransmit@28    10003044     winscard:WinSCard.dll
 0002:00000048       __imp__SCardStatusA@28     10003048     winscard:WinSCard.dll
 0002:0000004c       __imp__SCardEndTransaction@8 1000304c     winscard:WinSCard.dll
 0002:00000050       __imp__SCardBeginTransaction@4 10003050     winscard:WinSCard.dll
 0002:00000054       __imp__SCardControl@28     10003054     winscard:WinSCard.dll
 0002:00000058       __imp__SCardEstablishContext@16 10003058     winscard:WinSCard.dll
 0002:0000005c       __imp__SCardConnectA@24    1000305c     winscard:WinSCard.dll
 0002:00000060       __imp__SCardGetStatusChangeA@16 10003060     winscard:WinSCard.dll
 0002:00000064       __imp__SCardListReadersA@16 10003064     winscard:WinSCard.dll
 0002:00000068       __imp__SCardDisconnect@8   10003068     winscard:WinSCard.dll
 0002:0000006c       \177WinSCard_NULL_THUNK_DATA 1000306c     winscard:WinSCard.dll
 0002:00000070       __imp__free                10003070     ucrt:api-ms-win-crt-heap-l1-1-0.dll
 0002:00000074       __imp__malloc              10003074     ucrt:api-ms-win-crt-heap-l1-1-0.dll
 0002:00000078       __imp__calloc              10003078     ucrt:api-ms-win-crt-heap-l1-1-0.dll
 0002:0000007c       \177api-ms-win-crt-heap-l1-1-0_NULL_THUNK_DATA 1000307c     ucrt:api-ms-win-crt-heap-l1-1-0.dll
 0002:00000080       __imp___initterm           10003080     ucrt:api-ms-win-crt-runtime-l1-1-0.dll
 0002:00000084       __imp___initterm_e         10003084     ucrt:api-ms-win-crt-runtime-l1-1-0.dll
 0002:00000088       __imp___seh_filter_dll     10003088     ucrt:api-ms-win-crt-runtime-l1-1-0.dll
 0002:0000008c       __imp___configure_narrow_argv 1000308c     ucrt:api-ms-win-crt-runtime-l1-1-0.dll
 0002:00000090       __imp___initialize_narrow_environment 10003090     ucrt:api-ms-win-crt-runtime-l1-1-0.dll
 0002:00000094       __imp___initialize_onexit_table 10003094     ucrt:api-ms-win-crt-runtime-l1-1-0.dll
 0002:00000098       __imp___execute_onexit_table 10003098     ucrt:api-ms-win-crt-runtime-l1-1-0.dll
 0002:0000009c       __imp___cexit              1000309c     ucrt:api-ms-win-crt-runtime-l1-1-0.dll
 0002:000000a0       \177api-ms-win-crt-runtime-l1-1-0_NULL_THUNK_DATA 100030a0     ucrt:api-ms-win-crt-runtime-l1-1-0.dll
 0002:000000a4       __imp__strlen              100030a4     ucrt:api-ms-win-crt-string-l1-1-0.dll
 0002:000000a8       __imp__strdup              100030a8     ucrt:api-ms-win-crt-string-l1-1-0.dll
 0002:000000a8       __imp___strdup             100030a8     ucrt:api-ms-win-crt-string-l1-1-0.dll
 0002:000000ac       \177api-ms-win-crt-string-l1-1-0_NULL_THUNK_DATA 100030ac     ucrt:api-ms-win-crt-string-l1-1-0.dll
 0002:000000b0       ___guard_check_icall_fptr  100030b0     MSVCRT:guard_support.obj
 0002:000000b4       ___xc_a                    100030b4     MSVCRT:initializers.obj
 0002:000000b8       ___xc_z                    100030b8     MSVCRT:initializers.obj
 0002:000000bc       ___xi_a                    100030bc     MSVCRT:initializers.obj
 0002:000000c0       ___xi_z                    100030c0     MSVCRT:initializers.obj
 0002:000000c4       ___xp_a                    100030c4     MSVCRT:initializers.obj
 0002:000000c8       ___xp_z                    100030c8     MSVCRT:initializers.obj
 0002:000000cc       ___xt_a                    100030cc     MSVCRT:initializers.obj
 0002:000000d0       ___xt_z                    100030d0     MSVCRT:initializers.obj
 0002:000000d8       ??_C@_0BL@ENCPOIKC@java?1lang?1OutOfMemoryError@ 100030d8     pcsc.obj
 0002:000000f4       ??_C@_0CH@CNFHJICF@sun?1security?1smartcardio?1PCSCEx@ 100030f4     pcsc.obj
 0002:0000011c       ??_C@_04PFANPMCN@?$CII?$CJV@ 1000311c     pcsc.obj
 0002:00000124       ??_C@_06FALKBLGB@?$DMinit?$DO@ 10003124     pcsc.obj
 0002:0000012c       ??_C@_0BB@FLFAIHG@java?1lang?1String@ 1000312c     pcsc.obj
 0002:00000140       __pDefaultRawDllMain       10003140     MSVCRT:dll_dllmain.obj
 0002:00000140       __pRawDllMain              10003140     MSVCRT:dll_dllmain.obj
 0002:000001c0       __load_config_used         100031c0     MSVCRT:loadcfg.obj
 0002:00000278       ___safe_se_handler_table   10003278     <linker-defined>
 0002:00000500       ___rtc_iaa                 10003500     MSVCRT:initsect.obj
 0002:00000504       ___rtc_izz                 10003504     MSVCRT:initsect.obj
 0002:00000508       ___rtc_taa                 10003508     MSVCRT:initsect.obj
 0002:0000050c       ___rtc_tzz                 1000350c     MSVCRT:initsect.obj
 0002:00000880       __IMPORT_DESCRIPTOR_WinSCard 10003880     winscard:WinSCard.dll
 0002:00000894       __IMPORT_DESCRIPTOR_KERNEL32 10003894     kernel32:KERNEL32.dll
 0002:000008a8       __IMPORT_DESCRIPTOR_VCRUNTIME140 100038a8     vcruntime:VCRUNTIME140.dll
 0002:000008bc       __IMPORT_DESCRIPTOR_api-ms-win-crt-heap-l1-1-0 100038bc     ucrt:api-ms-win-crt-heap-l1-1-0.dll
 0002:000008d0       __IMPORT_DESCRIPTOR_api-ms-win-crt-string-l1-1-0 100038d0     ucrt:api-ms-win-crt-string-l1-1-0.dll
 0002:000008e4       __IMPORT_DESCRIPTOR_api-ms-win-crt-runtime-l1-1-0 100038e4     ucrt:api-ms-win-crt-runtime-l1-1-0.dll
 0002:000008f8       __NULL_IMPORT_DESCRIPTOR   100038f8     winscard:WinSCard.dll
 0003:00000000       ___security_cookie_complement 10004000     MSVCRT:gs_cookie.obj
 0003:00000004       ___security_cookie         10004004     MSVCRT:gs_cookie.obj
 0003:00000008       ___scrt_native_dllmain_reason 10004008     MSVCRT:utility.obj
 0003:00000010       ___isa_enabled             10004010     MSVCRT:cpu_disp.obj
 0003:00000014       ___scrt_ucrt_dll_is_in_use 10004014     MSVCRT:ucrt_stubs.obj
 0003:00000340       ?__type_info_root_node@@3U__type_info_node@@A 10004340     MSVCRT:tncleanup.obj
 0003:00000348       ?_OptionsStorage@?1??__local_stdio_printf_options@@9@4_KA 10004348     MSVCRT:default_local_stdio_options.obj
 0003:00000350       ?_OptionsStorage@?1??__local_stdio_scanf_options@@9@4_KA 10004350     MSVCRT:default_local_stdio_options.obj
 0003:00000358       ___scrt_current_native_startup_state 10004358     MSVCRT:utility.obj
 0003:0000035c       ___scrt_native_startup_lock 1000435c     MSVCRT:utility.obj
 0003:0000037c       ___scrt_debugger_hook_flag 1000437c     MSVCRT:utility_desktop.obj
 0003:00000380       ___isa_available           10004380     MSVCRT:cpu_disp.obj
 0003:00000384       ___favor                   10004384     MSVCRT:cpu_disp.obj
 0003:00000388       ___dyn_tls_init_callback   10004388     <common>

 entry point at        0001:00000b6d

 Static symbols

 0000:ffff9000       .debug$S                   10000000     j2pcsc.exp
 0000:ffff9000       .debug$S                   10000000     vcruntime:VCRUNTIME140.dll
 0000:ffff9000       .debug$S                   10000000     vcruntime:VCRUNTIME140.dll
 0000:ffff9000       .debug$S                   10000000     vcruntime:VCRUNTIME140.dll
 0000:ffff9000       .debug$S                   10000000     vcruntime:VCRUNTIME140.dll
 0000:ffff9000       .debug$S                   10000000     vcruntime:VCRUNTIME140.dll
 0000:ffff9000       .debug$S                   10000000     ucrt:api-ms-win-crt-heap-l1-1-0.dll
 0000:ffff9000       .debug$S                   10000000     ucrt:api-ms-win-crt-heap-l1-1-0.dll
 0000:ffff9000       .debug$S                   10000000     ucrt:api-ms-win-crt-heap-l1-1-0.dll
 0000:ffff9000       .debug$S                   10000000     ucrt:api-ms-win-crt-runtime-l1-1-0.dll
 0000:ffff9000       .debug$S                   10000000     ucrt:api-ms-win-crt-runtime-l1-1-0.dll
 0000:ffff9000       .debug$S                   10000000     ucrt:api-ms-win-crt-runtime-l1-1-0.dll
 0000:ffff9000       .debug$S                   10000000     ucrt:api-ms-win-crt-runtime-l1-1-0.dll
 0000:ffff9000       .debug$S                   10000000     ucrt:api-ms-win-crt-runtime-l1-1-0.dll
 0000:ffff9000       .debug$S                   10000000     ucrt:api-ms-win-crt-runtime-l1-1-0.dll
 0000:ffff9000       .debug$S                   10000000     ucrt:api-ms-win-crt-runtime-l1-1-0.dll
 0000:ffff9000       .debug$S                   10000000     ucrt:api-ms-win-crt-runtime-l1-1-0.dll
 0000:ffff9000       .debug$S                   10000000     ucrt:api-ms-win-crt-runtime-l1-1-0.dll
 0000:ffff9000       .debug$S                   10000000     ucrt:api-ms-win-crt-runtime-l1-1-0.dll
 0000:ffff9000       .debug$S                   10000000     ucrt:api-ms-win-crt-runtime-l1-1-0.dll
 0000:ffff9000       .debug$S                   10000000     ucrt:api-ms-win-crt-runtime-l1-1-0.dll
 0000:ffff9000       .debug$S                   10000000     ucrt:api-ms-win-crt-string-l1-1-0.dll
 0000:ffff9000       .debug$S                   10000000     ucrt:api-ms-win-crt-string-l1-1-0.dll
 0000:ffff9000       .debug$S                   10000000     kernel32:KERNEL32.dll
 0000:ffff9000       .debug$S                   10000000     kernel32:KERNEL32.dll
 0000:ffff9000       .debug$S                   10000000     kernel32:KERNEL32.dll
 0000:ffff9000       .debug$S                   10000000     kernel32:KERNEL32.dll
 0000:ffff9000       .debug$S                   10000000     kernel32:KERNEL32.dll
 0000:ffff9000       .debug$S                   10000000     kernel32:KERNEL32.dll
 0000:ffff9000       .debug$S                   10000000     kernel32:KERNEL32.dll
 0000:ffff9000       .debug$S                   10000000     kernel32:KERNEL32.dll
 0000:ffff9000       .debug$S                   10000000     kernel32:KERNEL32.dll
 0000:ffff9000       .debug$S                   10000000     kernel32:KERNEL32.dll
 0000:ffff9000       .debug$S                   10000000     kernel32:KERNEL32.dll
 0000:ffff9000       .debug$S                   10000000     kernel32:KERNEL32.dll
 0000:ffff9000       .debug$S                   10000000     kernel32:KERNEL32.dll
 0000:ffff9000       .debug$S                   10000000     kernel32:KERNEL32.dll
 0000:ffff9000       .debug$S                   10000000     winscard:WinSCard.dll
 0000:ffff9000       .debug$S                   10000000     winscard:WinSCard.dll
 0000:ffff9000       .debug$S                   10000000     winscard:WinSCard.dll
 0000:ffff9000       .debug$S                   10000000     winscard:WinSCard.dll
 0000:ffff9000       .debug$S                   10000000     winscard:WinSCard.dll
 0000:ffff9000       .debug$S                   10000000     winscard:WinSCard.dll
 0000:ffff9000       .debug$S                   10000000     winscard:WinSCard.dll
 0000:ffff9000       .debug$S                   10000000     winscard:WinSCard.dll
 0000:ffff9000       .debug$S                   10000000     winscard:WinSCard.dll
 0000:ffff9000       .debug$S                   10000000     winscard:WinSCard.dll
 0001:00000800       $$000000                   10001800     MSVCRT:chkstk.obj
 0001:0000082d       ?dllmain_crt_dispatch@@YGHQAUHINSTANCE__@@KQAX@Z 1000182d f   MSVCRT:dll_dllmain.obj
 0001:00000880       ?dllmain_crt_process_attach@@YAHQAUHINSTANCE__@@QAX@Z 10001880 f   MSVCRT:dll_dllmain.obj
 0001:00000987       ?dllmain_crt_process_detach@@YAH_N@Z 10001987 f   MSVCRT:dll_dllmain.obj
 0001:00000a37       ?dllmain_dispatch@@YAHQAUHINSTANCE__@@KQAX@Z 10001a37 f   MSVCRT:dll_dllmain.obj
 0001:00000b42       ?dllmain_raw@@YGHQAUHINSTANCE__@@KQAX@Z 10001b42 f   MSVCRT:dll_dllmain.obj
 0001:00000cb1       ___get_entropy             10001cb1 f   MSVCRT:gs_support.obj
 0001:00000dac       ?find_pe_section@@YAPAU_IMAGE_SECTION_HEADER@@QAEI@Z 10001dac f   MSVCRT:utility.obj
 0001:00001210       $$000000                   10002210     MSVCRT:sehprolg4.obj
 0002:00000144       _GS_ExceptionPointers      10003144     MSVCRT:gs_report.obj
 0002:00000510       __sehtable$?dllmain_crt_process_attach@@YAHQAUHINSTANCE__@@QAX@Z 10003510     MSVCRT:dll_dllmain.obj
 0002:00000530       __sehtable$?dllmain_crt_process_detach@@YAH_N@Z 10003530     MSVCRT:dll_dllmain.obj
 0002:00000558       __sehtable$?dllmain_dispatch@@YAHQAUHINSTANCE__@@KQAX@Z 10003558     MSVCRT:dll_dllmain.obj
 0002:00000578       __sehtable$___scrt_is_nonwritable_in_current_image 10003578     MSVCRT:utility.obj
 0002:000005a0       .edata                     100035a0     j2pcsc.exp
 0002:000005c8       rgpv                       100035c8     j2pcsc.exp
 0002:000005f4       rgszName                   100035f4     j2pcsc.exp
 0002:00000620       rgwOrd                     10003620     j2pcsc.exp
 0002:00000636       szName                     10003636     j2pcsc.exp
 0002:00000641       $N00001                    10003641     j2pcsc.exp
 0002:0000064f       $N00002                    1000364f     j2pcsc.exp
 0002:0000068c       $N00003                    1000368c     j2pcsc.exp
 0002:000006c0       $N00004                    100036c0     j2pcsc.exp
 0002:000006f4       $N00005                    100036f4     j2pcsc.exp
 0002:0000072b       $N00006                    1000372b     j2pcsc.exp
 0002:00000766       $N00007                    10003766     j2pcsc.exp
 0002:000007a3       $N00008                    100037a3     j2pcsc.exp
 0002:000007df       $N00009                    100037df     j2pcsc.exp
 0002:00000817       $N00010                    10003817     j2pcsc.exp
 0002:0000084a       $N00011                    1000384a     j2pcsc.exp
 0002:00000a80       .idata$6                   10003a80     winscard:WinSCard.dll
 0002:00000bb2       .idata$6                   10003bb2     kernel32:KERNEL32.dll
 0002:00000c04       .idata$6                   10003c04     vcruntime:VCRUNTIME140.dll
 0002:00000cec       .idata$6                   10003cec     ucrt:api-ms-win-crt-heap-l1-1-0.dll
 0002:00000d0c       .idata$6                   10003d0c     ucrt:api-ms-win-crt-string-l1-1-0.dll
 0002:00000d2e       .idata$6                   10003d2e     ucrt:api-ms-win-crt-runtime-l1-1-0.dll
 0003:00000018       ?__proc_attached@@3HA      10004018     MSVCRT:dll_dllmain.obj
 0003:00000020       _GS_ExceptionRecord        10004020     MSVCRT:gs_report.obj
 0003:00000070       _GS_ContextRecord          10004070     MSVCRT:gs_report.obj
 0003:00000360       ?is_initialized_as_dll@@3_NA 10004360     MSVCRT:utility.obj
 0003:00000361       ?module_local_atexit_table_initialized@@3_NA 10004361     MSVCRT:utility.obj
 0003:00000364       ?module_local_atexit_table@@3U_onexit_table_t@@A 10004364     MSVCRT:utility.obj
 0003:00000370       ?module_local_at_quick_exit_table@@3U_onexit_table_t@@A 10004370     MSVCRT:utility.obj
 0004:00000060       $R000000                   10005060     j2pcsc.dll.res
